:100000000C9434000C9446000C9446000C9446006A
:100010000C9446000C9446000C9446000C94460048
:100020000C9446000C9446000C9446000C94460038
:100030000C9446000C9446000C9446000C94460028
:100040000C9446000C9446000C9446000C94460018
:100050000C9446000C9446000C9446000C94460008
:100060000C9446000C94460011241FBECFEFD8E03C
:10007000DEBFCDBF11E0A0E0B1E001C01D92AE3007
:10008000B107E1F70E946C000C94F1010C940000A0
:10009000FC01A285B3858C9184FB222720F930E0F6
:1000A000318720870484F585E02D8081232B19F08A
:1000B0008460808308958B7F80830895229A25E24F
:1000C00030E0FC0135872487249823E230E0338731
:1000D000228780E090E00895CF92DF92EF92FF9226
:1000E00080E091E00E945E00C12CD12C760160E09E
:1000F00070E0CB01609300017093010180930201D5
:100100009093030180E091E00E9448008FEFC81AAD
:10011000D80AE80AF80AC701B6010E9400012FE6D2
:1001200032E143E05BE30E948E0120E030E0A90170
:100130000E949C00DFCF5058BB27AA270ED0B4C026
:10014000A5D030F0AAD020F031F49F3F11F41EF476
:100150009AC00EF4E095E7FB90C0E92FB6D080F38B
:10016000BA17620773078407950718F071F49EF5B4
:10017000CEC00EF4E0950B2EBA2FA02D0B01B901C5
:1001800090010C01CA01A0011124FF27591B99F00D
:10019000593F50F4503E68F11A16F040A22F232F19
:1001A000342F4427585FF3CF469537952795A79569
:1001B000F0405395C9F77EF41F16BA0B620B730B10
:1001C000840BBAF09150A1F0FF0FBB1F661F771F81
:1001D000881FC2F70EC0BA0F621F731F841F48F436
:1001E000879577956795B795F7959E3F08F0B3CFBC
:1001F0009395880F08F09927EE0F979587950895A6
:10020000E89409C097FB3EF49095809570956195B0
:100210007F4F8F4F9F4F9923A9F0F92F96E9BB2766
:100220009395F695879577956795B795F111F8CFE2
:10023000FAF4BB0F11F460FF1BC06F5F7F4F8F4F4D
:100240009F4F16C0882311F096E911C0772321F043
:100250009EE8872F762F05C0662371F096E8862FDB
:1002600070E060E02AF09A95660F771F881FDAF732
:10027000880F9695879597F9089597F99F6780E875
:1002800070E060E008959FEF80EC089500240A94E8
:100290001616170618060906089500240A94121661
:1002A0001306140605060895092E0394000C11F494
:1002B000882352F0BB0F40F4BF2B11F460FF04C041
:1002C0006F5F7F4F8F4F9F4F089557FD9058440F9A
:1002D000551F59F05F3F71F04795880F97FB991FA5
:1002E00061F09F3F79F08795089512161306140662
:1002F000551FF2CF4695F1DF08C0161617061806EF
:10030000991FF1CF86957105610508940895E894C9
:10031000BB2766277727CB0197F908950BD0C4CF69
:10032000B5DF28F0BADF18F0952309F0A6CFABCFE0
:100330001124EECFCADFA0F3959FD1F3950F50E0C3
:10034000551F629FF001729FBB27F00DB11D639F87
:10035000AA27F00DB11DAA1F649F6627B00DA11D2D
:10036000661F829F2227B00DA11D621F739FB00DD3
:10037000A11D621F839FA00D611D221F749F332743
:10038000A00D611D231F849F600D211D822F762FDC
:100390006A2F11249F5750408AF0E1F088234AF0D9
:1003A000EE0FFF1FBB1F661F771F881F9150504025
:1003B000A9F79E3F510570F060CFAACF5F3FECF3E5
:1003C000983EDCF3869577956795B795F795E79511
:1003D0009F5FC1F7FE2B880F911D9695879597F922
:0603E0000895F894FFCF20
:00000001FF
